 followref004

 Timestamp is a600f3ec (reproducible build file hash)

 Preferred load address is 0000000180000000

 Start         Length     Name                   Class
 0001:00000000 00003c20H .text$mn                CODE
 0001:00003c20 00000036H .text$mn$00             CODE
 0001:00003c56 00000092H .text$x                 CODE
 0002:00000000 000001c8H .idata$5                DATA
 0002:000001c8 00000038H .00cfg                  DATA
 0002:00000200 00000008H .CRT$XCA                DATA
 0002:00000208 00000008H .CRT$XCZ                DATA
 0002:00000210 00000008H .CRT$XIA                DATA
 0002:00000218 00000008H .CRT$XIC                DATA
 0002:00000220 00000008H .CRT$XIZ                DATA
 0002:00000228 00000008H .CRT$XLA                DATA
 0002:00000230 00000008H .CRT$XLZ                DATA
 0002:00000238 00000008H .CRT$XPA                DATA
 0002:00000240 00000008H .CRT$XPZ                DATA
 0002:00000248 00000008H .CRT$XTA                DATA
 0002:00000250 00000010H .CRT$XTZ                DATA
 0002:00000258 00000000H .gehcont$y              DATA
 0002:00000258 00000000H .gfids$y                DATA
 0002:00000260 00002320H .rdata                  DATA
 0002:00002580 00000000H .rdata$CastGuardVftablesA DATA
 0002:00002580 00000000H .rdata$CastGuardVftablesC DATA
 0002:00002580 00000028H .rdata$T                DATA
 0002:000025a8 000000bcH .rdata$voltmd           DATA
 0002:00002664 0000031cH .rdata$zzzdbg           DATA
 0002:00002980 00000008H .rtc$IAA                DATA
 0002:00002988 00000008H .rtc$IZZ                DATA
 0002:00002990 00000008H .rtc$TAA                DATA
 0002:00002998 00000008H .rtc$TZZ                DATA
 0002:000029a0 00000004H .tls                    DATA
 0002:000029a4 00000004H .tls$                   DATA
 0002:000029a8 00000008H .tls$ZZZ                DATA
 0002:000029b0 00000380H .xdata                  DATA
 0002:00002d30 00000364H .edata                  DATA
 0002:00003094 0000008cH .idata$2                DATA
 0002:00003120 00000018H .idata$3                DATA
 0002:00003138 000001c8H .idata$4                DATA
 0002:00003300 00000486H .idata$6                DATA
 0003:00000000 00000080H .data                   DATA
 0003:00000080 0001b2c8H .bss                    DATA
 0004:00000000 00000468H .pdata                  DATA

  Address         Publics by Value              Rva+Base               Lib:Object

 0000:00000000       __AbsoluteZero             0000000000000000     <absolute>
 0000:00000000       ___safe_se_handler_count   0000000000000000     <absolute>
 0000:00000000       ___safe_se_handler_table   0000000000000000     <absolute>
 0000:00000000       __arm64x_extra_rfe_table   0000000000000000     <absolute>
 0000:00000000       __arm64x_extra_rfe_table_size 0000000000000000     <absolute>
 0000:00000000       __arm64x_native_entrypoint 0000000000000000     <absolute>
 0000:00000000       __arm64x_redirection_metadata 0000000000000000     <absolute>
 0000:00000000       __arm64x_redirection_metadata_count 0000000000000000     <absolute>
 0000:00000000       __dynamic_value_reloc_table 0000000000000000     <absolute>
 0000:00000000       __enclave_config           0000000000000000     <absolute>
 0000:00000000       __guard_check_icall_a64n_fptr 0000000000000000     <absolute>
 0000:00000000       __guard_eh_cont_count      0000000000000000     <absolute>
 0000:00000000       __guard_eh_cont_table      0000000000000000     <absolute>
 0000:00000000       __guard_fids_count         0000000000000000     <absolute>
 0000:00000000       __guard_fids_table         0000000000000000     <absolute>
 0000:00000000       __guard_iat_count          0000000000000000     <absolute>
 0000:00000000       __guard_iat_table          0000000000000000     <absolute>
 0000:00000000       __guard_longjmp_count      0000000000000000     <absolute>
 0000:00000000       __guard_longjmp_table      0000000000000000     <absolute>
 0000:00000000       __hybrid_auxiliary_iat     0000000000000000     <absolute>
 0000:00000000       __hybrid_auxiliary_iat_copy 0000000000000000     <absolute>
 0000:00000000       __hybrid_code_map          0000000000000000     <absolute>
 0000:00000000       __hybrid_code_map_count    0000000000000000     <absolute>
 0000:00000000       __x64_code_ranges_to_entry_points 0000000000000000     <absolute>
 0000:00000000       __x64_code_ranges_to_entry_points_count 0000000000000000     <absolute>
 0000:00000100       __guard_flags              0000000000000100     <absolute>
 0000:00000000       __ImageBase                0000000180000000     <linker-defined>
 0001:00000000       ?NewObject@JNIEnv_@@QEAAPEAV_jobject@@PEAV_jclass@@PEAU_jmethodID@@ZZ 0000000180001000 f i libfollowref004.obj
 0001:00000028       ?TranslateError@@YAPEBDW4jvmtiError@@@Z 0000000180001028 f   libfollowref004.obj
 0001:000002e0       ?nsk_jni_check_exception@@YAHPEAUJNIEnv_@@QEBDH@Z 00000001800012e0 f   libfollowref004.obj
 0001:00000424       ?nsk_jni_lverify@@YAHHPEAUJNIEnv_@@HQEBDH1ZZ 0000000180001424 f   libfollowref004.obj
 0001:000004c4       Agent_Initialize           00000001800014c4 f   libfollowref004.obj
 0001:000006f4       Agent_OnAttach             00000001800016f4 f   libfollowref004.obj
 0001:000006f4       Agent_OnLoad               00000001800016f4 f   libfollowref004.obj
 0001:000006fc       Java_nsk_jvmti_unit_FollowReferences_FollowRefObjects_addRefToVerify 00000001800016fc f   libfollowref004.obj
 0001:000008d4       Java_nsk_jvmti_unit_FollowReferences_FollowRefObjects_getTag 00000001800018d4 f   libfollowref004.obj
 0001:00000994       Java_nsk_jvmti_unit_FollowReferences_FollowRefObjects_resetRefsToVerify 0000000180001994 f   libfollowref004.obj
 0001:0000099c       Java_nsk_jvmti_unit_FollowReferences_FollowRefObjects_resetTags 000000018000199c f   libfollowref004.obj
 0001:000009e0       Java_nsk_jvmti_unit_FollowReferences_FollowRefObjects_setTag 00000001800019e0 f   libfollowref004.obj
 0001:00000c38       Java_nsk_share_jvmti_ArgumentHandler_getAgentOptionsString 0000000180001c38 f   libfollowref004.obj
 0001:00000ce8       Java_nsk_share_jvmti_DebugeeClass_checkStatus 0000000180001ce8 f   libfollowref004.obj
 0001:00000d70       Java_nsk_share_jvmti_DebugeeClass_resetAgentData 0000000180001d70 f   libfollowref004.obj
 0001:00000dd0       Java_nsk_share_jvmti_RedefineAgent_agentStatus 0000000180001dd0 f   libfollowref004.obj
 0001:00000ddc       Java_nsk_share_jvmti_RedefineAgent_isRedefined 0000000180001ddc f   libfollowref004.obj
 0001:00000de8       Java_nsk_share_jvmti_RedefineAgent_redefineAttempted 0000000180001de8 f   libfollowref004.obj
 0001:00000df4       MA_checkStatus             0000000180001df4 f   libfollowref004.obj
 0001:00000e98       __local_stdio_printf_options 0000000180001e98 f i libfollowref004.obj
 0001:00001220       arrayPrimitiveValueCallback 0000000180002220 f   libfollowref004.obj
 0001:000012b4       checkThatAllTagsVisited    00000001800022b4 f   libfollowref004.obj
 0001:0000135c       checkUserData              000000018000235c f   libfollowref004.obj
 0001:000016fc       exitOnError                00000001800026fc f   libfollowref004.obj
 0001:000017b0       fprintf                    00000001800027b0 f i libfollowref004.obj
 0001:000017f4       heapReferenceCallback      00000001800027f4 f   libfollowref004.obj
 0001:000018c8       jvmti_FollowRefObject_init 00000001800028c8 f   libfollowref004.obj
 0001:00001924       markRefToVerify            0000000180002924 f   libfollowref004.obj
 0001:00001984       nsk_complain               0000000180002984 f   libfollowref004.obj
 0001:000019b0       nsk_jvmti_createJVMTIEnv   00000001800029b0 f   libfollowref004.obj
 0001:00001ae0       nsk_jvmti_lverify          0000000180002ae0 f   libfollowref004.obj
 0001:00001bd0       nsk_jvmti_parseOptions     0000000180002bd0 f   libfollowref004.obj
 0001:00001e20       nsk_jvmti_resetAgentData   0000000180002e20 f   libfollowref004.obj
 0001:00001ea0       nsk_jvmti_resumeSync       0000000180002ea0 f   libfollowref004.obj
 0001:00001f48       nsk_jvmti_setFailStatus    0000000180002f48 f   libfollowref004.obj
 0001:00001f84       nsk_jvmti_waitForSync      0000000180002f84 f   libfollowref004.obj
 0001:00002088       nsk_lcomplain              0000000180003088 f   libfollowref004.obj
 0001:000020a8       nsk_ldisplay               00000001800030a8 f   libfollowref004.obj
 0001:000020c8       nsk_ltrace                 00000001800030c8 f   libfollowref004.obj
 0001:000020e8       nsk_lvcomplain             00000001800030e8 f   libfollowref004.obj
 0001:000022a0       nsk_lvdisplay              00000001800032a0 f   libfollowref004.obj
 0001:000022ec       nsk_lverify                00000001800032ec f   libfollowref004.obj
 0001:00002348       nsk_lvtrace                0000000180003348 f   libfollowref004.obj
 0001:000023a8       nsk_printf                 00000001800033a8 f   libfollowref004.obj
 0001:000023d0       nsk_vprintf                00000001800033d0 f   libfollowref004.obj
 0001:00002484       primitiveFieldCallback     0000000180003484 f   libfollowref004.obj
 0001:00002520       printHeapRefCallbackInfo   0000000180003520 f   libfollowref004.obj
 0001:00002690       printf                     0000000180003690 f i libfollowref004.obj
 0001:00002a20       stringPrimitiveValueCallback 0000000180003a20 f   libfollowref004.obj
 0001:00002c14       wrongArrayPrimitiveValueCallback 0000000180003c14 f   libfollowref004.obj
 0001:00002c4c       wrongHeapReferenceCallback 0000000180003c4c f   libfollowref004.obj
 0001:00002c84       wrongPrimitiveFieldCallback 0000000180003c84 f   libfollowref004.obj
 0001:00002cbc       wrongStringPrimitiveValueCallback 0000000180003cbc f   libfollowref004.obj
 0001:00002cf4       __raise_securityfailure    0000000180003cf4 f   MSVCRT:gs_report.obj
 0001:00002d28       __report_gsfailure         0000000180003d28 f   MSVCRT:gs_report.obj
 0001:00002f68       __GSHandlerCheck           0000000180003f68 f   MSVCRT:gshandler.obj
 0001:00002f88       __GSHandlerCheckCommon     0000000180003f88 f   MSVCRT:gshandler.obj
 0001:00003000       __security_check_cookie    0000000180004000 f   MSVCRT:amdsecgs.obj
 0001:00003340       _DllMainCRTStartup         0000000180004340 f   MSVCRT:dll_dllmain.obj
 0001:00003380       __scrt_acquire_startup_lock 0000000180004380 f   MSVCRT:utility.obj
 0001:000033bc       __scrt_dllmain_after_initialize_c 00000001800043bc f   MSVCRT:utility.obj
 0001:000033f0       __scrt_dllmain_before_initialize_c 00000001800043f0 f   MSVCRT:utility.obj
 0001:00003408       __scrt_dllmain_crt_thread_attach 0000000180004408 f   MSVCRT:utility.obj
 0001:00003430       __scrt_dllmain_crt_thread_detach 0000000180004430 f   MSVCRT:utility.obj
 0001:00003448       __scrt_dllmain_exception_filter 0000000180004448 f   MSVCRT:utility.obj
 0001:000034a8       __scrt_dllmain_uninitialize_c 00000001800044a8 f   MSVCRT:utility.obj
 0001:000034d8       __scrt_dllmain_uninitialize_critical 00000001800044d8 f   MSVCRT:utility.obj
 0001:000034ec       __scrt_initialize_crt      00000001800044ec f   MSVCRT:utility.obj
 0001:00003538       __scrt_initialize_onexit_tables 0000000180004538 f   MSVCRT:utility.obj
 0001:000035c4       __scrt_is_nonwritable_in_current_image 00000001800045c4 f   MSVCRT:utility.obj
 0001:0000365c       __scrt_release_startup_lock 000000018000465c f   MSVCRT:utility.obj
 0001:00003680       __scrt_uninitialize_crt    0000000180004680 f   MSVCRT:utility.obj
 0001:000036ac       _onexit                    00000001800046ac f   MSVCRT:utility.obj
 0001:000036e8       atexit                     00000001800046e8 f   MSVCRT:utility.obj
 0001:00003700       __crt_debugger_hook        0000000180004700 f   MSVCRT:utility_desktop.obj
 0001:00003708       __scrt_fastfail            0000000180004708 f   MSVCRT:utility_desktop.obj
 0001:00003854       _guard_check_icall_nop     0000000180004854 f i MSVCRT:guard_support.obj
 0001:00003858       __security_init_cookie     0000000180004858 f   MSVCRT:gs_support.obj
 0001:00003904       DllMain                    0000000180004904 f   MSVCRT:dll_dllmain_stub.obj
 0001:00003928       ?__scrt_initialize_type_info@@YAXXZ 0000000180004928 f   MSVCRT:tncleanup.obj
 0001:00003938       ?__scrt_uninitialize_type_info@@YAXXZ 0000000180004938 f   MSVCRT:tncleanup.obj
 0001:00003944       __local_stdio_scanf_options 0000000180004944 f i MSVCRT:default_local_stdio_options.obj
 0001:0000394c       __scrt_initialize_default_local_stdio_options 000000018000494c f   MSVCRT:default_local_stdio_options.obj
 0001:00003968       __scrt_get_dyn_tls_init_callback 0000000180004968 f   MSVCRT:dyn_tls_init.obj
 0001:00003970       _RTC_Initialize            0000000180004970 f   MSVCRT:initsect.obj
 0001:000039ac       _RTC_Terminate             00000001800049ac f   MSVCRT:initsect.obj
 0001:000039e8       __isa_available_init       00000001800049e8 f   MSVCRT:cpu_disp.obj
 0001:00003b94       _get_startup_argv_mode     0000000180004b94 f   MSVCRT:argv_mode.obj
 0001:00003b9c       __scrt_is_ucrt_dll_in_use  0000000180004b9c f   MSVCRT:ucrt_detection.obj
 0001:00003bb0       memcpy                     0000000180004bb0 f   vcruntime:VCRUNTIME140.dll
 0001:00003bb6       memset                     0000000180004bb6 f   vcruntime:VCRUNTIME140.dll
 0001:00003bbc       strchr                     0000000180004bbc f   vcruntime:VCRUNTIME140.dll
 0001:00003bc2       __C_specific_handler       0000000180004bc2 f   vcruntime:VCRUNTIME140.dll
 0001:00003bc8       __std_type_info_destroy_list 0000000180004bc8 f   vcruntime:VCRUNTIME140.dll
 0001:00003bce       strcmp                     0000000180004bce f   ucrt:api-ms-win-crt-string-l1-1-0.dll
 0001:00003bd4       strlen                     0000000180004bd4 f   ucrt:api-ms-win-crt-string-l1-1-0.dll
 0001:00003bda       _initterm                  0000000180004bda f   ucrt:api-ms-win-crt-runtime-l1-1-0.dll
 0001:00003be0       _initterm_e                0000000180004be0 f   ucrt:api-ms-win-crt-runtime-l1-1-0.dll
 0001:00003be6       _seh_filter_dll            0000000180004be6 f   ucrt:api-ms-win-crt-runtime-l1-1-0.dll
 0001:00003bec       _configure_narrow_argv     0000000180004bec f   ucrt:api-ms-win-crt-runtime-l1-1-0.dll
 0001:00003bf2       _initialize_narrow_environment 0000000180004bf2 f   ucrt:api-ms-win-crt-runtime-l1-1-0.dll
 0001:00003bf8       _initialize_onexit_table   0000000180004bf8 f   ucrt:api-ms-win-crt-runtime-l1-1-0.dll
 0001:00003bfe       _register_onexit_function  0000000180004bfe f   ucrt:api-ms-win-crt-runtime-l1-1-0.dll
 0001:00003c04       _execute_onexit_table      0000000180004c04 f   ucrt:api-ms-win-crt-runtime-l1-1-0.dll
 0001:00003c0a       _crt_atexit                0000000180004c0a f   ucrt:api-ms-win-crt-runtime-l1-1-0.dll
 0001:00003c10       _cexit                     0000000180004c10 f   ucrt:api-ms-win-crt-runtime-l1-1-0.dll
 0001:00003c18       __acrt_initialize          0000000180004c18 f   MSVCRT:ucrt_stubs.obj
 0001:00003c18       __acrt_thread_attach       0000000180004c18 f   MSVCRT:ucrt_stubs.obj
 0001:00003c18       __acrt_thread_detach       0000000180004c18 f   MSVCRT:ucrt_stubs.obj
 0001:00003c18       __acrt_uninitialize        0000000180004c18 f   MSVCRT:ucrt_stubs.obj
 0001:00003c18       __acrt_uninitialize_critical 0000000180004c18 f   MSVCRT:ucrt_stubs.obj
 0001:00003c18       __scrt_stub_for_acrt_initialize 0000000180004c18 f   MSVCRT:ucrt_stubs.obj
 0001:00003c18       __scrt_stub_for_acrt_thread_attach 0000000180004c18 f   MSVCRT:ucrt_stubs.obj
 0001:00003c18       __scrt_stub_for_acrt_thread_detach 0000000180004c18 f   MSVCRT:ucrt_stubs.obj
 0001:00003c18       __scrt_stub_for_acrt_uninitialize 0000000180004c18 f   MSVCRT:ucrt_stubs.obj
 0001:00003c18       __scrt_stub_for_acrt_uninitialize_critical 0000000180004c18 f   MSVCRT:ucrt_stubs.obj
 0001:00003c18       __vcrt_initialize          0000000180004c18 f   MSVCRT:ucrt_stubs.obj
 0001:00003c18       __vcrt_thread_attach       0000000180004c18 f   MSVCRT:ucrt_stubs.obj
 0001:00003c18       __vcrt_thread_detach       0000000180004c18 f   MSVCRT:ucrt_stubs.obj
 0001:00003c18       __vcrt_uninitialize        0000000180004c18 f   MSVCRT:ucrt_stubs.obj
 0001:00003c18       __vcrt_uninitialize_critical 0000000180004c18 f   MSVCRT:ucrt_stubs.obj
 0001:00003c1c       __scrt_stub_for_is_c_termination_complete 0000000180004c1c f   MSVCRT:ucrt_stubs.obj
 0001:00003c1c       _is_c_termination_complete 0000000180004c1c f   MSVCRT:ucrt_stubs.obj
 0001:00003c30       _guard_dispatch_icall_nop  0000000180004c30 f   MSVCRT:guard_dispatch.obj
 0001:00003c50       _guard_xfg_dispatch_icall_nop 0000000180004c50 f   MSVCRT:guard_xfg_dispatch.obj
 0002:00000000       __imp_RtlCaptureContext    0000000180005000     kernel32:KERNEL32.dll
 0002:00000008       __imp_RtlLookupFunctionEntry 0000000180005008     kernel32:KERNEL32.dll
 0002:00000010       __imp_RtlVirtualUnwind     0000000180005010     kernel32:KERNEL32.dll
 0002:00000018       __imp_UnhandledExceptionFilter 0000000180005018     kernel32:KERNEL32.dll
 0002:00000020       __imp_SetUnhandledExceptionFilter 0000000180005020     kernel32:KERNEL32.dll
 0002:00000028       __imp_GetCurrentProcess    0000000180005028     kernel32:KERNEL32.dll
 0002:00000030       __imp_TerminateProcess     0000000180005030     kernel32:KERNEL32.dll
 0002:00000038       __imp_IsProcessorFeaturePresent 0000000180005038     kernel32:KERNEL32.dll
 0002:00000040       __imp_CloseHandle          0000000180005040     kernel32:KERNEL32.dll
 0002:00000048       __imp_InitializeCriticalSectionAndSpinCount 0000000180005048     kernel32:KERNEL32.dll
 0002:00000050       __imp_DeleteCriticalSection 0000000180005050     kernel32:KERNEL32.dll
 0002:00000058       __imp_CreateEventW         0000000180005058     kernel32:KERNEL32.dll
 0002:00000060       __imp_GetModuleHandleW     0000000180005060     kernel32:KERNEL32.dll
 0002:00000068       __imp_GetProcAddress       0000000180005068     kernel32:KERNEL32.dll
 0002:00000070       __imp_IsDebuggerPresent    0000000180005070     kernel32:KERNEL32.dll
 0002:00000078       __imp_QueryPerformanceCounter 0000000180005078     kernel32:KERNEL32.dll
 0002:00000080       __imp_GetCurrentProcessId  0000000180005080     kernel32:KERNEL32.dll
 0002:00000088       __imp_GetCurrentThreadId   0000000180005088     kernel32:KERNEL32.dll
 0002:00000090       __imp_GetSystemTimeAsFileTime 0000000180005090     kernel32:KERNEL32.dll
 0002:00000098       __imp_DisableThreadLibraryCalls 0000000180005098     kernel32:KERNEL32.dll
 0002:000000a0       __imp_InitializeSListHead  00000001800050a0     kernel32:KERNEL32.dll
 0002:000000a8       \177KERNEL32_NULL_THUNK_DATA 00000001800050a8     kernel32:KERNEL32.dll
 0002:000000b0       __imp_memcpy               00000001800050b0     vcruntime:VCRUNTIME140.dll
 0002:000000b8       __imp_memset               00000001800050b8     vcruntime:VCRUNTIME140.dll
 0002:000000c0       __imp_strchr               00000001800050c0     vcruntime:VCRUNTIME140.dll
 0002:000000c8       __imp___C_specific_handler 00000001800050c8     vcruntime:VCRUNTIME140.dll
 0002:000000d0       __imp___std_type_info_destroy_list 00000001800050d0     vcruntime:VCRUNTIME140.dll
 0002:000000d8       \177VCRUNTIME140_NULL_THUNK_DATA 00000001800050d8     vcruntime:VCRUNTIME140.dll
 0002:000000e0       __imp_strtol               00000001800050e0     ucrt:api-ms-win-crt-convert-l1-1-0.dll
 0002:000000e8       \177api-ms-win-crt-convert-l1-1-0_NULL_THUNK_DATA 00000001800050e8     ucrt:api-ms-win-crt-convert-l1-1-0.dll
 0002:000000f0       __imp_malloc               00000001800050f0     ucrt:api-ms-win-crt-heap-l1-1-0.dll
 0002:000000f8       __imp_free                 00000001800050f8     ucrt:api-ms-win-crt-heap-l1-1-0.dll
 0002:00000100       \177api-ms-win-crt-heap-l1-1-0_NULL_THUNK_DATA 0000000180005100     ucrt:api-ms-win-crt-heap-l1-1-0.dll
 0002:00000108       __imp__errno               0000000180005108     ucrt:api-ms-win-crt-runtime-l1-1-0.dll
 0002:00000110       __imp_exit                 0000000180005110     ucrt:api-ms-win-crt-runtime-l1-1-0.dll
 0002:00000118       __imp__cexit               0000000180005118     ucrt:api-ms-win-crt-runtime-l1-1-0.dll
 0002:00000120       __imp__crt_atexit          0000000180005120     ucrt:api-ms-win-crt-runtime-l1-1-0.dll
 0002:00000128       __imp__execute_onexit_table 0000000180005128     ucrt:api-ms-win-crt-runtime-l1-1-0.dll
 0002:00000130       __imp__register_onexit_function 0000000180005130     ucrt:api-ms-win-crt-runtime-l1-1-0.dll
 0002:00000138       __imp__initialize_onexit_table 0000000180005138     ucrt:api-ms-win-crt-runtime-l1-1-0.dll
 0002:00000140       __imp__initialize_narrow_environment 0000000180005140     ucrt:api-ms-win-crt-runtime-l1-1-0.dll
 0002:00000148       __imp__configure_narrow_argv 0000000180005148     ucrt:api-ms-win-crt-runtime-l1-1-0.dll
 0002:00000150       __imp__seh_filter_dll      0000000180005150     ucrt:api-ms-win-crt-runtime-l1-1-0.dll
 0002:00000158       __imp__initterm_e          0000000180005158     ucrt:api-ms-win-crt-runtime-l1-1-0.dll
 0002:00000160       __imp__initterm            0000000180005160     ucrt:api-ms-win-crt-runtime-l1-1-0.dll
 0002:00000168       \177api-ms-win-crt-runtime-l1-1-0_NULL_THUNK_DATA 0000000180005168     ucrt:api-ms-win-crt-runtime-l1-1-0.dll
 0002:00000170       __imp___acrt_iob_func      0000000180005170     ucrt:api-ms-win-crt-stdio-l1-1-0.dll
 0002:00000178       __imp_fflush               0000000180005178     ucrt:api-ms-win-crt-stdio-l1-1-0.dll
 0002:00000180       __imp___stdio_common_vsprintf 0000000180005180     ucrt:api-ms-win-crt-stdio-l1-1-0.dll
 0002:00000188       __imp___stdio_common_vfprintf 0000000180005188     ucrt:api-ms-win-crt-stdio-l1-1-0.dll
 0002:00000190       \177api-ms-win-crt-stdio-l1-1-0_NULL_THUNK_DATA 0000000180005190     ucrt:api-ms-win-crt-stdio-l1-1-0.dll
 0002:00000198       __imp_strcmp               0000000180005198     ucrt:api-ms-win-crt-string-l1-1-0.dll
 0002:000001a0       __imp__strdup              00000001800051a0     ucrt:api-ms-win-crt-string-l1-1-0.dll
 0002:000001a0       __imp_strdup               00000001800051a0     ucrt:api-ms-win-crt-string-l1-1-0.dll
 0002:000001a8       __imp_strlen               00000001800051a8     ucrt:api-ms-win-crt-string-l1-1-0.dll
 0002:000001b0       __imp_strpbrk              00000001800051b0     ucrt:api-ms-win-crt-string-l1-1-0.dll
 0002:000001b8       __imp_strncpy              00000001800051b8     ucrt:api-ms-win-crt-string-l1-1-0.dll
 0002:000001c0       \177api-ms-win-crt-string-l1-1-0_NULL_THUNK_DATA 00000001800051c0     ucrt:api-ms-win-crt-string-l1-1-0.dll
 0002:000001c8       __guard_check_icall_fptr   00000001800051c8     MSVCRT:guard_support.obj
 0002:000001d0       __guard_xfg_check_icall_fptr 00000001800051d0     MSVCRT:guard_support.obj
 0002:000001d8       __guard_dispatch_icall_fptr 00000001800051d8     MSVCRT:guard_support.obj
 0002:000001e0       __guard_xfg_dispatch_icall_fptr 00000001800051e0     MSVCRT:guard_support.obj
 0002:000001e8       __guard_xfg_table_dispatch_icall_fptr 00000001800051e8     MSVCRT:guard_support.obj
 0002:000001f0       __castguard_check_failure_os_handled_fptr 00000001800051f0     MSVCRT:guard_support.obj
 0002:000001f8       __guard_memcpy_fptr        00000001800051f8     vcruntime:softmemtag.obj
 0002:00000200       __xc_a                     0000000180005200     MSVCRT:initializers.obj
 0002:00000208       __xc_z                     0000000180005208     MSVCRT:initializers.obj
 0002:00000210       __xi_a                     0000000180005210     MSVCRT:initializers.obj
 0002:00000220       __xi_z                     0000000180005220     MSVCRT:initializers.obj
 0002:00000228       __xl_a                     0000000180005228     MSVCRT:tlssup.obj
 0002:00000230       __xl_z                     0000000180005230     MSVCRT:tlssup.obj
 0002:00000238       __xp_a                     0000000180005238     MSVCRT:initializers.obj
 0002:00000240       __xp_z                     0000000180005240     MSVCRT:initializers.obj
 0002:00000248       __xt_a                     0000000180005248     MSVCRT:initializers.obj
 0002:00000250       __xt_z                     0000000180005250     MSVCRT:initializers.obj
 0002:00000260       g_refKindStr               0000000180005260     libfollowref004.obj
 0002:00000410       ??_C@_09BPLDFGCI@unknown_0@ 0000000180005410     libfollowref004.obj
 0002:00000420       ??_C@_0BL@FPNMECJD@JVMTI_HEAP_REFERENCE_CLASS@ 0000000180005420     libfollowref004.obj
 0002:00000440       ??_C@_0BL@FKGKKLNM@JVMTI_HEAP_REFERENCE_FIELD@ 0000000180005440     libfollowref004.obj
 0002:00000460       ??_C@_0CD@CAEHCFJF@JVMTI_HEAP_REFERENCE_ARRAY_ELEM@ 0000000180005460     libfollowref004.obj
 0002:00000488       ??_C@_0CC@DNEBMCNK@JVMTI_HEAP_REFERENCE_CLASS_LOAD@ 0000000180005488     libfollowref004.obj
 0002:000004b0       ??_C@_0BN@CJMIPEBB@JVMTI_HEAP_REFERENCE_SIGNERS@ 00000001800054b0     libfollowref004.obj
 0002:000004d0       ??_C@_0CH@HBOIDPEB@JVMTI_HEAP_REFERENCE_PROTECTION@ 00000001800054d0     libfollowref004.obj
 0002:000004f8       ??_C@_0BP@MDKGDGKL@JVMTI_HEAP_REFERENCE_INTERFACE@ 00000001800054f8     libfollowref004.obj
 0002:00000518       ??_C@_0CC@JJMIHNJH@JVMTI_HEAP_REFERENCE_STATIC_FIE@ 0000000180005518     libfollowref004.obj
 0002:00000540       ??_C@_0CD@IDHEEGID@JVMTI_HEAP_REFERENCE_CONSTANT_P@ 0000000180005540     libfollowref004.obj
 0002:00000568       ??_C@_0CA@EFFCHNG@JVMTI_HEAP_REFERENCE_SUPERCLASS@ 0000000180005568     libfollowref004.obj
 0002:00000588       ??_C@_0L@PCDFHGCJ@unknown_11@ 0000000180005588     libfollowref004.obj
 0002:00000598       ??_C@_0L@NJBICFOK@unknown_12@ 0000000180005598     libfollowref004.obj
 0002:000005a8       ??_C@_0L@MAADBEKL@unknown_13@ 00000001800055a8     libfollowref004.obj
 0002:000005b8       ??_C@_0L@IPECICGM@unknown_14@ 00000001800055b8     libfollowref004.obj
 0002:000005c8       ??_C@_0L@JGFJLDCN@unknown_15@ 00000001800055c8     libfollowref004.obj
 0002:000005d8       ??_C@_0L@LNHEOAOO@unknown_16@ 00000001800055d8     libfollowref004.obj
 0002:000005e8       ??_C@_0L@KEGPNBKP@unknown_17@ 00000001800055e8     libfollowref004.obj
 0002:000005f8       ??_C@_0L@CDPHMNGA@unknown_18@ 00000001800055f8     libfollowref004.obj
 0002:00000608       ??_C@_0L@DKOMPMCB@unknown_19@ 0000000180005608     libfollowref004.obj
 0002:00000618       ??_C@_0L@OJGIPJDB@unknown_20@ 0000000180005618     libfollowref004.obj
 0002:00000628       ??_C@_0CA@KAOFNDEM@JVMTI_HEAP_REFERENCE_JNI_GLOBAL@ 0000000180005628     libfollowref004.obj
 0002:00000648       ??_C@_0CC@HPFAJBK@JVMTI_HEAP_REFERENCE_SYSTEM_CLA@ 0000000180005648     libfollowref004.obj
 0002:00000670       ??_C@_0BN@FDEGFOHC@JVMTI_HEAP_REFERENCE_MONITOR@ 0000000180005670     libfollowref004.obj
 0002:00000690       ??_C@_0CB@HKIBCMAJ@JVMTI_HEAP_REFERENCE_STACK_LOCA@ 0000000180005690     libfollowref004.obj
 0002:000006b8       ??_C@_0BP@EAACMMOE@JVMTI_HEAP_REFERENCE_JNI_LOCAL@ 00000001800056b8     libfollowref004.obj
 0002:000006d8       ??_C@_0BM@IJDEOGOE@JVMTI_HEAP_REFERENCE_THREAD@ 00000001800056d8     libfollowref004.obj
 0002:000006f8       ??_C@_0BL@EDGPPKC@JVMTI_HEAP_REFERENCE_OTHER@ 00000001800056f8     libfollowref004.obj
 0002:00000714       ??_C@_04BCJPDBDA@Code@     0000000180005714     libfollowref004.obj
 0002:00000720       ??_C@_0BA@OCLMCFKC@LineNumberTable@ 0000000180005720     libfollowref004.obj
 0002:00000730       ??_C@_0BD@CPAEPILC@LocalVariableTable@ 0000000180005730     libfollowref004.obj
 0002:00000748       ??_C@_0BH@NMBDNHBD@LocalVariableTypeTable@ 0000000180005748     libfollowref004.obj
 0002:00000760       ??_C@_0O@HIHEEDNJ@StackMapTable@ 0000000180005760     libfollowref004.obj
 0002:00000770       ??_C@_0L@HCDIAMJG@?9?5?$CFs?0?5?$CFd?3?5@ 0000000180005770     libfollowref004.obj
 0002:00000780       ??_C@_0JI@HLPECLFI@?$CD?5?4?4?4?6?$CD?5ERROR?3?5too?5many?5complai@ 0000000180005780     libfollowref004.obj
 0002:00000820       ??_C@_0ED@JNEKCCOB@The?5following?5fake?5exception?5st@ 0000000180005820     libfollowref004.obj
 0002:00000868       ??_C@_0CN@FCNMDFBH@nsk?4share?4Fake_Exception_for_RU@ 0000000180005868     libfollowref004.obj
 0002:00000898       ??_C@_08PGFFNAEI@?$CI?$CFs?3?$CFd?$CJ?5@ 0000000180005898     libfollowref004.obj
 0002:000008a8       ??_C@_0DP@IENMAEGI@s?2test?2hotspot?2jtreg?2vmTestbase@ 00000001800058a8     libfollowref004.obj
 0002:000008e8       ??_C@_0BL@NDJLFFJB@?7at?5nsk_lvcomplain?$CI?$CFs?3?$CFd?$CJ?6@ 00000001800058e8     libfollowref004.obj
 0002:00000908       ??_C@_0BC@JOOKAFKF@?$CD?5ERROR?3?5?$CFs?0?5?$CFd?3?5@ 0000000180005908     libfollowref004.obj
 0002:00000920       ??_C@_09KJEAHMEH@?$CD?5ERROR?3?5@ 0000000180005920     libfollowref004.obj
 0002:0000092c       ??_C@_02GPIOPFAK@?$DO?$DO@ 000000018000592c     libfollowref004.obj
 0002:00000930       ??_C@_02FODMEDOG@?$DM?$DM@ 0000000180005930     libfollowref004.obj
 0002:00000934       ??_C@_02DJGKEECL@?4?4@     0000000180005934     libfollowref004.obj
 0002:00000938       ??_C@_0O@CJPGJOAF@?9?5?$CFs?0?5?$CFd?3?5?$CFs?5@ 0000000180005938     libfollowref004.obj
 0002:00000948       ??_C@_0CB@IAKPDOIC@?$CD?5?5?5verified?5assertion?5is?5FALSE@ 0000000180005948     libfollowref004.obj
 0002:00000970       ??_C@_0CO@LGONDEPD@stdout?3?5fflush?5failed?5?9?5err?$DN?$CFd?5@ 0000000180005970     libfollowref004.obj
 0002:000009a0       ??_C@_0CO@KBGKJPBD@stderr?3?5fflush?5failed?5?9?5err?$DN?$CFd?5@ 00000001800059a0     libfollowref004.obj
 0002:000009d0       ??_C@_06PAOMPDJH@?$DMnone?$DO@ 00000001800059d0     libfollowref004.obj
 0002:000009d8       ??_C@_0BB@JCNMKLLK@JVMTI_ERROR_NONE@ 00000001800059d8     libfollowref004.obj
 0002:000009f0       ??_C@_0BL@LDIMKLPH@JVMTI_ERROR_INVALID_THREAD@ 00000001800059f0     libfollowref004.obj
 0002:00000a10       ??_C@_0CB@PJFPAIKJ@JVMTI_ERROR_INVALID_THREAD_GROU@ 0000000180005a10     libfollowref004.obj
 0002:00000a38       ??_C@_0BN@LLMKHMNF@JVMTI_ERROR_INVALID_PRIORITY@ 0000000180005a38     libfollowref004.obj
 0002:00000a58       ??_C@_0CB@MBOFKAGB@JVMTI_ERROR_THREAD_NOT_SUSPENDE@ 0000000180005a58     libfollowref004.obj
 0002:00000a80       ??_C@_0BN@FABOLPBI@JVMTI_ERROR_THREAD_SUSPENDED@ 0000000180005a80     libfollowref004.obj
 0002:00000aa0       ??_C@_0BN@FDGNOBJM@JVMTI_ERROR_THREAD_NOT_ALIVE@ 0000000180005aa0     libfollowref004.obj
 0002:00000ac0       ??_C@_0BL@GOBIFKNJ@JVMTI_ERROR_INVALID_OBJECT@ 0000000180005ac0     libfollowref004.obj
 0002:00000ae0       ??_C@_0BK@FCMAJPPC@JVMTI_ERROR_INVALID_CLASS@ 0000000180005ae0     libfollowref004.obj
 0002:00000b00       ??_C@_0BP@IKLLBKEB@JVMTI_ERROR_CLASS_NOT_PREPARED@ 0000000180005b00     libfollowref004.obj
 0002:00000b20       ??_C@_0BN@KLPPLKG@JVMTI_ERROR_INVALID_METHODID@ 0000000180005b20     libfollowref004.obj
 0002:00000b40       ??_C@_0BN@BCEKOKND@JVMTI_ERROR_INVALID_LOCATION@ 0000000180005b40     libfollowref004.obj
 0002:00000b60       ??_C@_0BM@DFDGPME@JVMTI_ERROR_INVALID_FIELDID@ 0000000180005b60     libfollowref004.obj
 0002:00000b80       ??_C@_0BL@NELIEPEC@JVMTI_ERROR_NO_MORE_FRAMES@ 0000000180005b80     libfollowref004.obj
 0002:00000ba0       ??_C@_0BJ@BDBECFDM@JVMTI_ERROR_OPAQUE_FRAME@ 0000000180005ba0     libfollowref004.obj
 0002:00000bc0       ??_C@_0BK@MIIFNLOB@JVMTI_ERROR_TYPE_MISMATCH@ 0000000180005bc0     libfollowref004.obj
 0002:00000be0       ??_C@_0BJ@HPCAOILC@JVMTI_ERROR_INVALID_SLOT@ 0000000180005be0     libfollowref004.obj
 0002:00000c00       ??_C@_0BG@CHILOPNI@JVMTI_ERROR_DUPLICATE@ 0000000180005c00     libfollowref004.obj
 0002:00000c18       ??_C@_0BG@DIEMLHKM@JVMTI_ERROR_NOT_FOUND@ 0000000180005c18     libfollowref004.obj
 0002:00000c30       ??_C@_0BM@NHMCKHOB@JVMTI_ERROR_INVALID_MONITOR@ 0000000180005c30     libfollowref004.obj
 0002:00000c50       ??_C@_0BO@PPEDAJGL@JVMTI_ERROR_NOT_MONITOR_OWNER@ 0000000180005c50     libfollowref004.obj
 0002:00000c70       ??_C@_0BG@FCAIPEID@JVMTI_ERROR_INTERRUPT@ 0000000180005c70     libfollowref004.obj
 0002:00000c88       ??_C@_0CB@EGDBNKOI@JVMTI_ERROR_INVALID_CLASS_FORMA@ 0000000180005c88     libfollowref004.obj
 0002:00000cb0       ??_C@_0CG@DGKOGIAL@JVMTI_ERROR_CIRCULAR_CLASS_DEFI@ 0000000180005cb0     libfollowref004.obj
 0002:00000cd8       ??_C@_0BP@ICEALPKC@JVMTI_ERROR_FAILS_VERIFICATION@ 0000000180005cd8     libfollowref004.obj
 0002:00000cf8       ??_C@_0DC@JDACLMIO@JVMTI_ERROR_UNSUPPORTED_REDEFIN@ 0000000180005cf8     libfollowref004.obj
 0002:00000d30       ??_C@_0DE@GKDKNOMJ@JVMTI_ERROR_UNSUPPORTED_REDEFIN@ 0000000180005d30     libfollowref004.obj
 0002:00000d68       ??_C@_0BO@LAFKIOG@JVMTI_ERROR_INVALID_TYPESTATE@ 0000000180005d68     libfollowref004.obj
 0002:00000d88       ??_C@_0DH@INDGCLLB@JVMTI_ERROR_UNSUPPORTED_REDEFIN@ 0000000180005d88     libfollowref004.obj
 0002:00000dc0       ??_C@_0DE@NHEOMMGI@JVMTI_ERROR_UNSUPPORTED_REDEFIN@ 0000000180005dc0     libfollowref004.obj
 0002:00000df8       ??_C@_0CA@EKPNJOEP@JVMTI_ERROR_UNSUPPORTED_VERSION@ 0000000180005df8     libfollowref004.obj
 0002:00000e18       ??_C@_0BN@OFFMAHHL@JVMTI_ERROR_NAMES_DONT_MATCH@ 0000000180005e18     libfollowref004.obj
 0002:00000e38       ??_C@_0DN@HHBBLAKE@JVMTI_ERROR_UNSUPPORTED_REDEFIN@ 0000000180005e38     libfollowref004.obj
 0002:00000e78       ??_C@_0DO@HMBGBGNA@JVMTI_ERROR_UNSUPPORTED_REDEFIN@ 0000000180005e78     libfollowref004.obj
 0002:00000eb8       ??_C@_0BP@PBECGKHJ@JVMTI_ERROR_UNMODIFIABLE_CLASS@ 0000000180005eb8     libfollowref004.obj
 0002:00000ed8       ??_C@_0BK@CANILEHF@JVMTI_ERROR_NOT_AVAILABLE@ 0000000180005ed8     libfollowref004.obj
 0002:00000ef8       ??_C@_0CE@INJKMEFK@JVMTI_ERROR_MUST_POSSESS_CAPABI@ 0000000180005ef8     libfollowref004.obj
 0002:00000f20       ??_C@_0BJ@LBFPFPDM@JVMTI_ERROR_NULL_POINTER@ 0000000180005f20     libfollowref004.obj
 0002:00000f40       ??_C@_0BP@CHJPNNEM@JVMTI_ERROR_ABSENT_INFORMATION@ 0000000180005f40     libfollowref004.obj
 0002:00000f60       ??_C@_0BP@OMFMNLC@JVMTI_ERROR_INVALID_EVENT_TYPE@ 0000000180005f60     libfollowref004.obj
 0002:00000f80       ??_C@_0BN@BIBNPHHO@JVMTI_ERROR_ILLEGAL_ARGUMENT@ 0000000180005f80     libfollowref004.obj
 0002:00000fa0       ??_C@_0BK@KKNDHDCE@JVMTI_ERROR_NATIVE_METHOD@ 0000000180005fa0     libfollowref004.obj
 0002:00000fc0       ??_C@_0BK@PMKCFHAE@JVMTI_ERROR_OUT_OF_MEMORY@ 0000000180005fc0     libfollowref004.obj
 0002:00000fe0       ??_C@_0BK@NNJBDMNB@JVMTI_ERROR_ACCESS_DENIED@ 0000000180005fe0     libfollowref004.obj
 0002:00001000       ??_C@_0BI@GHECLMNC@JVMTI_ERROR_WRONG_PHASE@ 0000000180006000     libfollowref004.obj
 0002:00001018       ??_C@_0BF@OLIHJOII@JVMTI_ERROR_INTERNAL@ 0000000180006018     libfollowref004.obj
 0002:00001030       ??_C@_0BO@EOHGKJHI@JVMTI_ERROR_UNATTACHED_THREAD@ 0000000180006030     libfollowref004.obj
 0002:00001050       ??_C@_0CA@LKHFDACL@JVMTI_ERROR_INVALID_ENVIRONMENT@ 0000000180006050     libfollowref004.obj
 0002:00001070       ??_C@_0BA@MMFHLOKK@?$DMunknown?5error?$DO@ 0000000180006070     libfollowref004.obj
 0002:00001080       ??_C@_0CF@CBHOKDB@throwable?5?$DN?5jni?9?$DOExceptionOccur@ 0000000180006080     libfollowref004.obj
 0002:000010a8       ??_C@_03OFAPEBGM@?$CFs?6@  00000001800060a8     libfollowref004.obj
 0002:000010b0       ??_C@_0DM@LPIGEGNJ@s?2test?2hotspot?2jtreg?2vmTestbase@ 00000001800060b0     libfollowref004.obj
 0002:000010f0       ??_C@_0CC@NFCNPEPK@Exception?5in?5JNI?5call?5?$CIcleared?$CJ@ 00000001800060f0     libfollowref004.obj
 0002:00001118       ??_C@_0BJ@IBAKFIKF@jni?9?$DOExceptionDescribe?$CI?$CJ@ 0000000180006118     libfollowref004.obj
 0002:00001138       ??_C@_0BG@GGKALKMH@jni?9?$DOExceptionClear?$CI?$CJ@ 0000000180006138     libfollowref004.obj
 0002:00001150       ??_C@_0CF@JMGFGJLJ@?$CD?5?5?5verified?5JNI?5assertion?5is?5F@ 0000000180006150     libfollowref004.obj
 0002:00001178       ??_C@_07KBAMPNJK@verbose@  0000000180006178     libfollowref004.obj
 0002:00001180       ??_C@_0DN@PKJBOLAP@nsk_jvmti_parseOptions?$CI?$CJ?3?5unexp@ 0000000180006180     libfollowref004.obj
 0002:000011c0       ??_C@_05IMBNNINJ@trace@    00000001800061c0     libfollowref004.obj
 0002:000011c8       ??_C@_0DD@BJKGNDMB@nsk_jvmti_parseOptions?$CI?$CJ?3?5no?5va@ 00000001800061c8     libfollowref004.obj
 0002:000011fc       ??_C@_04CGFJFPFD@none@     00000001800061fc     libfollowref004.obj
 0002:00001204       ??_C@_06BMELKFMA@before@   0000000180006204     libfollowref004.obj
 0002:0000120c       ??_C@_05CMKPCFDK@after@    000000018000620c     libfollowref004.obj
 0002:00001214       ??_C@_03NFKEKGGK@all@      0000000180006214     libfollowref004.obj
 0002:00001218       ??_C@_0DM@NDNJGJKE@nsk_jvmti_parseOptions?$CI?$CJ?3?5uexpe@ 0000000180006218     libfollowref004.obj
 0002:00001258       ??_C@_08NBBJKJO@waittime@  0000000180006258     libfollowref004.obj
 0002:00001268       ??_C@_0DO@CMHGAOHC@nsk_jvmti_parseOptions?$CI?$CJ?3?5not?5i@ 0000000180006268     libfollowref004.obj
 0002:000012a8       ??_C@_0DL@LNMPBDLN@nsk_jvmti_parseOptions?$CI?$CJ?3?5negat@ 00000001800062a8     libfollowref004.obj
 0002:000012e8       ??_C@_0DA@GMFJNOJH@nsk_jvmti_parseOptions?$CI?$CJ?3?5unkno@ 00000001800062e8     libfollowref004.obj
 0002:00001318       ??_C@_0CO@CCIAMEAN@nsk_jvmti_parseOptions?$CI?$CJ?3?5found@ 0000000180006318     libfollowref004.obj
 0002:00001348       ??_C@_0CJ@OEGPCGDL@nsk_jvmti_parseOptions?$CI?$CJ?3?5out?5o@ 0000000180006348     libfollowref004.obj
 0002:00001378       ??_C@_0DI@NMBHPGGF@nsk_jvmti_parseOptions?$CI?$CJ?3?5too?5m@ 0000000180006378     libfollowref004.obj
 0002:000013b0       ??_C@_03POGCGECB@?5?0?$HO@ 00000001800063b0     libfollowref004.obj
 0002:000013b8       ??_C@_0CB@MLNJNCLJ@?5?5jvmti?5error?3?5code?$DN?$CFd?0?5name?$DN?$CFs@ 00000001800063b8     libfollowref004.obj
 0002:000013e0       ??_C@_0CD@OHBGDKMK@?$CD?5?5?5jvmti?5error?3?5code?$DN?$CFd?0?5name?$DN@ 00000001800063e0     libfollowref004.obj
 0002:00001408       ??_C@_0CG@JNNCGPHB@?$CD?5?5?5error?5expected?3?5code?$DN?$CFd?0?5na@ 0000000180006408     libfollowref004.obj
 0002:00001430       ??_C@_0EB@IMGKPCGE@?$CIstr_obj?5?$DN?5jni?9?$DONewStringUTF?$CIco@ 0000000180006430     libfollowref004.obj
 0002:00001480       ??_C@_0EA@HFOGGBCC@s?2test?2hotspot?2jtreg?2vmTestbase@ 0000000180006480     libfollowref004.obj
 0002:000014c0       ??_C@_05KKCIMGE@error@     00000001800064c0     libfollowref004.obj
 0002:000014c8       ??_C@_0CJ@JACLEAA@Test?5failed?5by?5setFailStatus?$CI?$CJ?4@ 00000001800064c8     libfollowref004.obj
 0002:000014f8       ??_C@_0BD@HGNAOMCP@agent_data_monitor@ 00000001800064f8     libfollowref004.obj
 0002:00001510       ??_C@_0EB@OGCLGKLN@javaVM?9?$DOGetEnv?$CI?$CIvoid?5?$CK?$CK?$CJ?$CGjvmti_@ 0000000180006510     libfollowref004.obj
 0002:00001560       ??_C@_0EA@PNBCDMOA@s?2test?2hotspot?2jtreg?2vmTestbase@ 0000000180006560     libfollowref004.obj
 0002:000015a0       ??_C@_0CI@DDPIFBGM@init_agent_data?$CIjvmti_env?0?5?$CGage@ 00000001800065a0     libfollowref004.obj
 0002:000015c8       ??_C@_0DI@ILAHDLMP@?$CI?$CKagentThreadProc?$CJ?$CIjvmti_env?0?5a@ 00000001800065c8     libfollowref004.obj
 0002:00001600       ??_C@_0BD@KDBALNLB@JVMTI?5agent?5thread@ 0000000180006600     libfollowref004.obj
 0002:00001618       ??_C@_0BB@NOKBFPFO@java?1lang?1Thread@ 0000000180006618     libfollowref004.obj
 0002:0000162c       ??_C@_06FALKBLGB@?$DMinit?$DO@ 000000018000662c     libfollowref004.obj
 0002:00001638       ??_C@_0BG@IKDDPPGD@?$CILjava?1lang?1String?$DL?$CJV@ 0000000180006638     libfollowref004.obj
 0002:00001650       ??_C@_0EB@IFJBFEKC@?$CIthreadClass?5?$DN?5jni_env?9?$DOFindCla@ 0000000180006650     libfollowref004.obj
 0002:000016a0       ??_C@_0GF@FGFIBKKL@?$CIthreadCtor?5?$DN?5jni_env?9?$DOGetMetho@ 00000001800066a0     libfollowref004.obj
 0002:00001708       ??_C@_0DN@NCPDJLOG@?$CIthreadName?5?$DN?5jni_env?9?$DONewStrin@ 0000000180006708     libfollowref004.obj
 0002:00001750       ??_C@_0FE@PFKODBGC@?$CIthreadObject?5?$DN?5jni_env?9?$DONewObj@ 0000000180006750     libfollowref004.obj
 0002:000017b0       ??_C@_0ED@HOBAHHJI@?$CIthreadGlobalRef?5?$DN?5jni_env?9?$DONew@ 00000001800067b0     libfollowref004.obj
 0002:00001800       ??_C@_0FN@HNJJAHFC@jvmti_env?9?$DORunAgentThread?$CIagent@ 0000000180006800     libfollowref004.obj
 0002:00001860       ??_C@_0EA@MOJDNKDF@Debuggee?5status?5sync?5aborted?5be@ 0000000180006860     libfollowref004.obj
 0002:000018a0       ??_C@_0CO@PGPGMHBJ@No?5status?5sync?5occured?5for?5time@ 00000001800068a0     libfollowref004.obj
 0002:000018d0       ??_C@_0CL@DOEBDPKJ@Debuggee?5was?5not?5suspended?5on?5s@ 00000001800068d0     libfollowref004.obj
 0002:00001900       ??_C@_0EA@EEOEJAEN@status?5?$DN?5syncDebuggeeStatus?$CIjni@ 0000000180006900     libfollowref004.obj
 0002:00001940       ??_C@_0BL@JBCFNBMB@nsk_jvmti_resetAgentData?$CI?$CJ@ 0000000180006940     libfollowref004.obj
 0002:00001960       ??_C@_0CO@EPEAMNOL@Checking?5that?5all?5set?5tags?5have@ 0000000180006960     libfollowref004.obj
 0002:00001990       ??_C@_0EL@LPBEELIP@s?2test?2hotspot?2jtreg?2vmTestbase@ 0000000180006990     libfollowref004.obj
 0002:000019e0       ??_C@_0CE@EHHMKJPF@Tag?5?$CFI64d?5has?5not?5been?5visited?3@ 00000001800069e0     libfollowref004.obj
 0002:00001a08       ??_C@_0CN@IGHKFJNO@?$DO?$DO?$DO?5Tag?5?$CFI64d?5has?5been?5visited?5@ 0000000180006a08     libfollowref004.obj
 0002:00001a38       ??_C@_0CK@JDAMFDMJ@jvmti?9?$DOSetTag?$CIo?0?5tag?$CJ?5?$DN?$DN?5JVMTI_@ 0000000180006a38     libfollowref004.obj
 0002:00001a68       ??_C@_0CC@DAMNHKNI@Can?8t?5set?5tag?5?$CFli?5for?5object?5?$CFl@ 0000000180006a68     libfollowref004.obj
 0002:00001a90       ??_C@_0DL@HAJPNKEF@jvmti?9?$DOGetObjectHashCode?$CIo?0?5?$CGha@ 0000000180006a90     libfollowref004.obj
 0002:00001ad0       ??_C@_0BL@JFPIEOBF@Can?8t?5get?5hash?5object?5?$CFlx?6@ 0000000180006ad0     libfollowref004.obj
 0002:00001af0       ??_C@_0BG@DICPHBKN@setTag?3?5?$CF08x?5?$DM?9?5?$CF?53li@ 0000000180006af0     libfollowref004.obj
 0002:00001b08       ??_C@_0DH@FCEEBDMJ@?$CIs?5?$DN?5jni?9?$DOGetStringUTFChars?$CIsIn@ 0000000180006b08     libfollowref004.obj
 0002:00001b40       ??_C@_0BJ@OKKGHDCN@Can?8t?5get?5string?5at?5?$CF?$CDp?6@ 0000000180006b40     libfollowref004.obj
 0002:00001b60       ??_C@_0BP@EKFLGGFJ@Can?8t?5get?5string?5at?5?$CF?$CDp?3?5null?6@ 0000000180006b60     libfollowref004.obj
 0002:00001b80       ??_C@_06ICODBHCL@?5?1?1?5?$CFs@ 0000000180006b80     libfollowref004.obj
 0002:00001b88       ??_C@_0DB@KGFPLEGO@?$CIr?5?$DN?5jvmti?9?$DOGetTag?$CIo?0?5?$CGtag?$CJ?$CJ?5?$DN?$DN@ 0000000180006b88     libfollowref004.obj
 0002:00001bc0       ??_C@_0CO@PDAGBCGJ@Can?8t?5GetTag?5for?5object?5?$CFlx?4?5Re@ 0000000180006bc0     libfollowref004.obj
 0002:00001bf0       ??_C@_0CH@HPEODOHC@TEST_BUG?3?5Max?4?5number?5of?5refs?5r@ 0000000180006bf0     libfollowref004.obj
 0002:00001c18       ??_C@_0DI@PHFCABIM@?$CIr?5?$DN?5jvmti?9?$DOGetTag?$CIfrom?0?5?$CGtagFr@ 0000000180006c18     libfollowref004.obj
 0002:00001c50       ??_C@_0DI@MDEGFNKD@TEST_BUG?3?5Can?8t?5GetTag?5for?5obje@ 0000000180006c50     libfollowref004.obj
 0002:00001c88       ??_C@_0DE@MLELJAHM@?$CIr?5?$DN?5jvmti?9?$DOGetTag?$CIto?0?5?$CGtagTo?$CJ?$CJ@ 0000000180006c88     libfollowref004.obj
 0002:00001cc0       ??_C@_0HC@NNDCODGA@?$CFs?0?5?$CFi?3?5Unexpected?5user_data?5is@ 0000000180006cc0     libfollowref004.obj
 0002:00001d38       ??_C@_0BK@PFJCLOAC@heapReferenceCallback?3?5?$CFs@ 0000000180006d38     libfollowref004.obj
 0002:00001d60       ??_C@_0EI@NKIKAIHO@?5?5?5reference_info?3?5?$CF?$CDlx?0?5class_@ 0000000180006d60     libfollowref004.obj
 0002:00001db0       ??_C@_0ED@MFAGKNKA@?5?5?5size?3?5?$CFI64d?0?5tag_ptr?3?5?$CFp?0?5?5r@ 0000000180006db0     libfollowref004.obj
 0002:00001df8       ??_C@_0CE@GABMPACP@?5?5?5tag?3?5?$CFI64d?0?5referrer_tag?3?5?$CFI@ 0000000180006df8     libfollowref004.obj
 0002:00001e20       ??_C@_0BK@GKOJAMMG@?5?5?5summary?3?5?$CFs?3?5?$CFs?5?$DM?9?5?$CFs?6@ 0000000180006e20     libfollowref004.obj
 0002:00001e40       ??_C@_0DM@KOCHIMGJ@heap?5reference?5callback?5was?5cal@ 0000000180006e40     libfollowref004.obj
 0002:00001e80       ??_C@_0DN@BEPFBLJE@primitive?5field?5callback?5was?5ca@ 0000000180006e80     libfollowref004.obj
 0002:00001ec0       ??_C@_0ED@EJACFPJG@array?5primitive?5value?5callback?5@ 0000000180006ec0     libfollowref004.obj
 0002:00001f10       ??_C@_0EE@MIHJIODF@string?5primitive?5value?5callback@ 0000000180006f10     libfollowref004.obj
 0002:00001f60       ??_C@_0FO@EOCGJNJH@s?2test?2hotspot?2jtreg?2vmTestbase@ 0000000180006f60     libfollowref004.obj
 0002:00001fc0       ??_C@_0EG@EIHEEGH@?5primitiveFieldCallback?3?5ref?$DN?$CFs@ 0000000180006fc0     libfollowref004.obj
 0002:00002010       ??_C@_0EO@HJLHKNAC@?5?5?5?5arrayPrimitiveValueCallback@ 0000000180007010     libfollowref004.obj
 0002:00002060       ??_C@_0EC@DNGCCNKG@stringPrimitiveValueCallback?3?5c@ 0000000180007060     libfollowref004.obj
 0002:000020b0       ??_C@_0EB@PJFFFPOL@?$CIklass?5?$DN?5jni?9?$DOFindClass?$CIJAVA_LA@ 00000001800070b0     libfollowref004.obj
 0002:000020f8       ??_C@_0BB@FLFAIHG@java?1lang?1String@ 00000001800070f8     libfollowref004.obj
 0002:00002110       ??_C@_0DH@IFMJHGC@?$CIg_jniGlobalRef?5?$DN?5jni?9?$DONewGloba@ 0000000180007110     libfollowref004.obj
 0002:00002148       ??_C@_0DP@CDPIPACE@?$CIg_jniWeakGlobalRef?5?$DN?5jni?9?$DONewW@ 0000000180007148     libfollowref004.obj
 0002:00002188       ??_C@_0BJ@HFLGIHKK@?$DO?$DO?$DO?5Sync?5with?5Java?5code?6@ 0000000180007188     libfollowref004.obj
 0002:000021a8       ??_C@_0CB@JPBPHGGJ@nsk_jvmti_waitForSync?$CIg_timeout@ 00000001800071a8     libfollowref004.obj
 0002:000021d0       ??_C@_0CC@DPCJEPGM@?$DO?$DO?$DO?5Create?5JNI?5global?5reference@ 00000001800071d0     libfollowref004.obj
 0002:000021f8       ??_C@_0BM@HNAFBIHC@retCode?5?$DN?$DN?5JVMTI_ERROR_NONE@ 00000001800071f8     libfollowref004.obj
 0002:00002218       ??_C@_0BL@JFJNOPCD@?$DO?$DO?$DO?5Let?5debugee?5to?5finish?6@ 0000000180007218     libfollowref004.obj
 0002:00002238       ??_C@_0BH@LECMGIIA@nsk_jvmti_resumeSync?$CI?$CJ@ 0000000180007238     libfollowref004.obj
 0002:00002250       ??_C@_0CA@MNKGCBCG@nsk_jvmti_parseOptions?$CIoptions?$CJ@ 0000000180007250     libfollowref004.obj
 0002:00002270       ??_C@_0DN@MIAMNFPH@?$CIjvmti?5?$DN?5nsk_jvmti_createJVMTIE@ 0000000180007270     libfollowref004.obj
 0002:000022b0       ??_C@_0BO@DBKDIPGD@jvmti?9?$DOAddCapabilities?$CI?$CGcaps?$CJ@ 00000001800072b0     libfollowref004.obj
 0002:000022d0       ??_C@_0CL@PIACJIPK@nsk_jvmti_setAgentProc?$CIagentPro@ 00000001800072d0     libfollowref004.obj
 0002:00002310       ??_C@_1EC@JIJBPKFM@?$AAa?$AAp?$AAi?$AA?9?$AAm?$AAs?$AA?9?$AAw?$AAi?$AAn?$AA?9?$AAc?$AAo?$AAr?$AAe@ 0000000180007310     MSVCRT:thread_safe_statics.obj
 0002:00002358       ??_C@_1BK@MGMFAEKH@?$AAk?$AAe?$AAr?$AAn?$AAe?$AAl?$AA3?$AA2?$AA?4?$AAd?$AAl?$AAl@ 0000000180007358     MSVCRT:thread_safe_statics.obj
 0002:00002378       ??_C@_0BJ@JEBJOJFJ@SleepConditionVariableCS@ 0000000180007378     MSVCRT:thread_safe_statics.obj
 0002:00002398       ??_C@_0BJ@PGPPEPCC@WakeAllConditionVariable@ 0000000180007398     MSVCRT:thread_safe_statics.obj
 0002:000023b8       _pDefaultRawDllMain        00000001800073b8     MSVCRT:dll_dllmain.obj
 0002:000023b8       _pRawDllMain               00000001800073b8     MSVCRT:dll_dllmain.obj
 0002:000023c0       __xmm@ffffffffffffffffffffffffffffffff 00000001800073c0     MSVCRT:utility.obj
 0002:000023d0       _load_config_used          00000001800073d0     MSVCRT:loadcfg.obj
 0002:00002580       _tls_used                  0000000180007580     MSVCRT:tlssup.obj
 0002:000025a8       __volatile_metadata        00000001800075a8     <linker-defined>
 0002:00002980       __rtc_iaa                  0000000180007980     MSVCRT:initsect.obj
 0002:00002988       __rtc_izz                  0000000180007988     MSVCRT:initsect.obj
 0002:00002990       __rtc_taa                  0000000180007990     MSVCRT:initsect.obj
 0002:00002998       __rtc_tzz                  0000000180007998     MSVCRT:initsect.obj
 0002:000029a0       _tls_start                 00000001800079a0     MSVCRT:tlssup.obj
 0002:000029a4       _Init_thread_epoch         00000001800079a4     MSVCRT:thread_safe_statics.obj
 0002:000029a8       _tls_end                   00000001800079a8     MSVCRT:tlssup.obj
 0002:00003094       __IMPORT_DESCRIPTOR_KERNEL32 0000000180008094     kernel32:KERNEL32.dll
 0002:000030a8       __IMPORT_DESCRIPTOR_VCRUNTIME140 00000001800080a8     vcruntime:VCRUNTIME140.dll
 0002:000030bc       __IMPORT_DESCRIPTOR_api-ms-win-crt-heap-l1-1-0 00000001800080bc     ucrt:api-ms-win-crt-heap-l1-1-0.dll
 0002:000030d0       __IMPORT_DESCRIPTOR_api-ms-win-crt-runtime-l1-1-0 00000001800080d0     ucrt:api-ms-win-crt-runtime-l1-1-0.dll
 0002:000030e4       __IMPORT_DESCRIPTOR_api-ms-win-crt-convert-l1-1-0 00000001800080e4     ucrt:api-ms-win-crt-convert-l1-1-0.dll
 0002:000030f8       __IMPORT_DESCRIPTOR_api-ms-win-crt-stdio-l1-1-0 00000001800080f8     ucrt:api-ms-win-crt-stdio-l1-1-0.dll
 0002:0000310c       __IMPORT_DESCRIPTOR_api-ms-win-crt-string-l1-1-0 000000018000810c     ucrt:api-ms-win-crt-string-l1-1-0.dll
 0002:00003120       __NULL_IMPORT_DESCRIPTOR   0000000180008120     kernel32:KERNEL32.dll
 0003:00000030       _Init_global_epoch         0000000180009030     MSVCRT:thread_safe_statics.obj
 0003:00000040       __security_cookie          0000000180009040     MSVCRT:gs_cookie.obj
 0003:00000048       __security_cookie_complement 0000000180009048     MSVCRT:gs_cookie.obj
 0003:00000050       __scrt_native_dllmain_reason 0000000180009050     MSVCRT:utility.obj
 0003:00000058       __isa_available            0000000180009058     MSVCRT:cpu_disp.obj
 0003:0000005c       __isa_enabled              000000018000905c     MSVCRT:cpu_disp.obj
 0003:00000060       __memset_fast_string_threshold 0000000180009060     MSVCRT:cpu_disp.obj
 0003:00000068       __memset_nt_threshold      0000000180009068     MSVCRT:cpu_disp.obj
 0003:00000070       __scrt_ucrt_dll_is_in_use  0000000180009070     MSVCRT:ucrt_stubs.obj
 0003:00000080       g_wrongHeapCallbacks       0000000180009080     libfollowref004.obj
 0003:00000100       g_szTagInfo                0000000180009100     libfollowref004.obj
 0003:00002040       g_tagFlags                 000000018000b040     libfollowref004.obj
 0003:00002428       g_refsToVerifyCnt          000000018000b428     libfollowref004.obj
 0003:0000242c       g_fakeUserData             000000018000b42c     libfollowref004.obj
 0003:00002430       g_tagVisitCount            000000018000b430     libfollowref004.obj
 0003:000033d0       g_refsToVerify             000000018000c3d0     libfollowref004.obj
 0003:0001aad0       g_userDataError            0000000180023ad0     libfollowref004.obj
 0003:0001ad00       ?_OptionsStorage@?1??__local_stdio_printf_options@@9@4_KA 0000000180023d00     libfollowref004.obj
 0003:0001b2c8       _tls_index                 00000001800242c8     MSVCRT:tlssup.obj
 0003:0001b2d0       __scrt_current_native_startup_state 00000001800242d0     MSVCRT:utility.obj
 0003:0001b2d8       __scrt_native_startup_lock 00000001800242d8     MSVCRT:utility.obj
 0003:0001b318       __scrt_debugger_hook_flag  0000000180024318     MSVCRT:utility_desktop.obj
 0003:0001b320       ?__type_info_root_node@@3U__type_info_node@@A 0000000180024320     MSVCRT:tncleanup.obj
 0003:0001b330       ?_OptionsStorage@?1??__local_stdio_scanf_options@@9@4_KA 0000000180024330     MSVCRT:default_local_stdio_options.obj
 0003:0001b338       __favor                    0000000180024338     MSVCRT:cpu_disp.obj
 0003:0001b340       __dyn_tls_init_callback    0000000180024340     <common>

 entry point at        0001:00003340

 Static symbols

 0000:fffd9000       .debug$S                   0000000180000000     followref004.exp
 0000:fffd9000       .debug$S                   0000000180000000     vcruntime:VCRUNTIME140.dll
 0000:fffd9000       .debug$S                   0000000180000000     vcruntime:VCRUNTIME140.dll
 0000:fffd9000       .debug$S                   0000000180000000     vcruntime:VCRUNTIME140.dll
 0000:fffd9000       .debug$S                   0000000180000000     vcruntime:VCRUNTIME140.dll
 0000:fffd9000       .debug$S                   0000000180000000     vcruntime:VCRUNTIME140.dll
 0000:fffd9000       .debug$S                   0000000180000000     vcruntime:VCRUNTIME140.dll
 0000:fffd9000       .debug$S                   0000000180000000     vcruntime:VCRUNTIME140.dll
 0000:fffd9000       .debug$S                   0000000180000000     ucrt:api-ms-win-crt-convert-l1-1-0.dll
 0000:fffd9000       .debug$S                   0000000180000000     ucrt:api-ms-win-crt-heap-l1-1-0.dll
 0000:fffd9000       .debug$S                   0000000180000000     ucrt:api-ms-win-crt-heap-l1-1-0.dll
 0000:fffd9000       .debug$S                   0000000180000000     ucrt:api-ms-win-crt-heap-l1-1-0.dll
 0000:fffd9000       .debug$S                   0000000180000000     ucrt:api-ms-win-crt-heap-l1-1-0.dll
 0000:fffd9000       .debug$S                   0000000180000000     ucrt:api-ms-win-crt-runtime-l1-1-0.dll
 0000:fffd9000       .debug$S                   0000000180000000     ucrt:api-ms-win-crt-runtime-l1-1-0.dll
 0000:fffd9000       .debug$S                   0000000180000000     ucrt:api-ms-win-crt-runtime-l1-1-0.dll
 0000:fffd9000       .debug$S                   0000000180000000     ucrt:api-ms-win-crt-runtime-l1-1-0.dll
 0000:fffd9000       .debug$S                   0000000180000000     ucrt:api-ms-win-crt-runtime-l1-1-0.dll
 0000:fffd9000       .debug$S                   0000000180000000     ucrt:api-ms-win-crt-runtime-l1-1-0.dll
 0000:fffd9000       .debug$S                   0000000180000000     ucrt:api-ms-win-crt-runtime-l1-1-0.dll
 0000:fffd9000       .debug$S                   0000000180000000     ucrt:api-ms-win-crt-runtime-l1-1-0.dll
 0000:fffd9000       .debug$S                   0000000180000000     ucrt:api-ms-win-crt-runtime-l1-1-0.dll
 0000:fffd9000       .debug$S                   0000000180000000     ucrt:api-ms-win-crt-runtime-l1-1-0.dll
 0000:fffd9000       .debug$S                   0000000180000000     ucrt:api-ms-win-crt-runtime-l1-1-0.dll
 0000:fffd9000       .debug$S                   0000000180000000     ucrt:api-ms-win-crt-runtime-l1-1-0.dll
 0000:fffd9000       .debug$S                   0000000180000000     ucrt:api-ms-win-crt-runtime-l1-1-0.dll
 0000:fffd9000       .debug$S                   0000000180000000     ucrt:api-ms-win-crt-runtime-l1-1-0.dll
 0000:fffd9000       .debug$S                   0000000180000000     ucrt:api-ms-win-crt-runtime-l1-1-0.dll
 0000:fffd9000       .debug$S                   0000000180000000     ucrt:api-ms-win-crt-runtime-l1-1-0.dll
 0000:fffd9000       .debug$S                   0000000180000000     ucrt:api-ms-win-crt-stdio-l1-1-0.dll
 0000:fffd9000       .debug$S                   0000000180000000     ucrt:api-ms-win-crt-stdio-l1-1-0.dll
 0000:fffd9000       .debug$S                   0000000180000000     ucrt:api-ms-win-crt-stdio-l1-1-0.dll
 0000:fffd9000       .debug$S                   0000000180000000     ucrt:api-ms-win-crt-stdio-l1-1-0.dll
 0000:fffd9000       .debug$S                   0000000180000000     ucrt:api-ms-win-crt-stdio-l1-1-0.dll
 0000:fffd9000       .debug$S                   0000000180000000     ucrt:api-ms-win-crt-stdio-l1-1-0.dll
 0000:fffd9000       .debug$S                   0000000180000000     ucrt:api-ms-win-crt-stdio-l1-1-0.dll
 0000:fffd9000       .debug$S                   0000000180000000     ucrt:api-ms-win-crt-stdio-l1-1-0.dll
 0000:fffd9000       .debug$S                   0000000180000000     ucrt:api-ms-win-crt-stdio-l1-1-0.dll
 0000:fffd9000       .debug$S                   0000000180000000     ucrt:api-ms-win-crt-stdio-l1-1-0.dll
 0000:fffd9000       .debug$S                   0000000180000000     ucrt:api-ms-win-crt-string-l1-1-0.dll
 0000:fffd9000       .debug$S                   0000000180000000     ucrt:api-ms-win-crt-string-l1-1-0.dll
 0000:fffd9000       .debug$S                   0000000180000000     ucrt:api-ms-win-crt-string-l1-1-0.dll
 0000:fffd9000       .debug$S                   0000000180000000     ucrt:api-ms-win-crt-string-l1-1-0.dll
 0000:fffd9000       .debug$S                   0000000180000000     ucrt:api-ms-win-crt-string-l1-1-0.dll
 0000:fffd9000       .debug$S                   0000000180000000     ucrt:api-ms-win-crt-string-l1-1-0.dll
 0000:fffd9000       .debug$S                   0000000180000000     ucrt:api-ms-win-crt-string-l1-1-0.dll
 0000:fffd9000       .debug$S                   0000000180000000     ucrt:api-ms-win-crt-string-l1-1-0.dll
 0000:fffd9000       .debug$S                   0000000180000000     kernel32:KERNEL32.dll
 0000:fffd9000       .debug$S                   0000000180000000     kernel32:KERNEL32.dll
 0000:fffd9000       .debug$S                   0000000180000000     kernel32:KERNEL32.dll
 0000:fffd9000       .debug$S                   0000000180000000     kernel32:KERNEL32.dll
 0000:fffd9000       .debug$S                   0000000180000000     kernel32:KERNEL32.dll
 0000:fffd9000       .debug$S                   0000000180000000     kernel32:KERNEL32.dll
 0000:fffd9000       .debug$S                   0000000180000000     kernel32:KERNEL32.dll
 0000:fffd9000       .debug$S                   0000000180000000     kernel32:KERNEL32.dll
 0000:fffd9000       .debug$S                   0000000180000000     kernel32:KERNEL32.dll
 0000:fffd9000       .debug$S                   0000000180000000     kernel32:KERNEL32.dll
 0000:fffd9000       .debug$S                   0000000180000000     kernel32:KERNEL32.dll
 0000:fffd9000       .debug$S                   0000000180000000     kernel32:KERNEL32.dll
 0000:fffd9000       .debug$S                   0000000180000000     kernel32:KERNEL32.dll
 0000:fffd9000       .debug$S                   0000000180000000     kernel32:KERNEL32.dll
 0000:fffd9000       .debug$S                   0000000180000000     kernel32:KERNEL32.dll
 0000:fffd9000       .debug$S                   0000000180000000     kernel32:KERNEL32.dll
 0000:fffd9000       .debug$S                   0000000180000000     kernel32:KERNEL32.dll
 0000:fffd9000       .debug$S                   0000000180000000     kernel32:KERNEL32.dll
 0000:fffd9000       .debug$S                   0000000180000000     kernel32:KERNEL32.dll
 0000:fffd9000       .debug$S                   0000000180000000     kernel32:KERNEL32.dll
 0000:fffd9000       .debug$S                   0000000180000000     kernel32:KERNEL32.dll
 0000:fffd9000       .debug$S                   0000000180000000     kernel32:KERNEL32.dll
 0000:fffd9000       .debug$S                   0000000180000000     kernel32:KERNEL32.dll
 0000:fffd9000       .debug$S                   0000000180000000     kernel32:KERNEL32.dll
 0000:fffd9000       .debug$S                   0000000180000000     kernel32:KERNEL32.dll
 0000:fffd9000       .debug$S                   0000000180000000     kernel32:KERNEL32.dll
 0000:fffd9000       .debug$S                   0000000180000000     kernel32:KERNEL32.dll
 0000:fffd9000       .debug$S                   0000000180000000     kernel32:KERNEL32.dll
 0001:00000ea0       addRefToVerify             0000000180001ea0 f   libfollowref004.obj
 0001:00000f0c       agentProc                  0000000180001f0c f   libfollowref004.obj
 0001:000010b4       agentThreadWrapper         00000001800020b4 f   libfollowref004.obj
 0001:000013ac       check_option               00000001800023ac f   libfollowref004.obj
 0001:00001570       createGlobalRefs           0000000180002570 f   libfollowref004.obj
 0001:00001780       file_basename              0000000180002780 f   libfollowref004.obj
 0001:000026e0       startAgentThreadWrapper    00000001800036e0 f   libfollowref004.obj
 0001:00002a7c       syncDebuggeeStatus         0000000180003a7c f   libfollowref004.obj
 0001:00002dfc       capture_previous_context   0000000180003dfc f   MSVCRT:gs_report.obj
 0001:00002e70       ?__scrt_initialize_thread_safe_statics@@YAHXZ 0000000180003e70 f   MSVCRT:thread_safe_statics.obj
 0001:00002f40       ?__scrt_uninitialize_thread_safe_statics@@YAXXZ 0000000180003f40 f   MSVCRT:thread_safe_statics.obj
 0001:00002ff0       $$000000                   0000000180003ff0     MSVCRT:amdsecgs.obj
 0001:00003020       ?dllmain_crt_dispatch@@YAHQEAUHINSTANCE__@@KQEAX@Z 0000000180004020 f   MSVCRT:dll_dllmain.obj
 0001:00003070       ?dllmain_crt_process_attach@@YAHQEAUHINSTANCE__@@QEAX@Z 0000000180004070 f   MSVCRT:dll_dllmain.obj
 0001:00003188       ?dllmain_crt_process_detach@@YAH_N@Z 0000000180004188 f   MSVCRT:dll_dllmain.obj
 0001:0000320c       ?dllmain_dispatch@@YAHQEAUHINSTANCE__@@KQEAX@Z 000000018000420c f   MSVCRT:dll_dllmain.obj
 0001:00003c20       $$000000                   0000000180004c20     MSVCRT:guard_dispatch.obj
 0001:00003c40       $$000000                   0000000180004c40     MSVCRT:guard_xfg_dispatch.obj
 0001:00003c56       ?fin$0@?0??dllmain_crt_process_attach@@YAHQEAUHINSTANCE__@@QEAX@Z@4HA 0000000180004c56 f   MSVCRT:dll_dllmain.obj
 0001:00003c6d       ?fin$0@?0??dllmain_crt_process_detach@@YAH_N@Z@4HA 0000000180004c6d f   MSVCRT:dll_dllmain.obj
 0001:00003c86       ?fin$1@?0??dllmain_crt_process_detach@@YAH_N@Z@4HA 0000000180004c86 f   MSVCRT:dll_dllmain.obj
 0001:00003c9a       ?filt$0@?0??dllmain_dispatch@@YAHQEAUHINSTANCE__@@KQEAX@Z@4HA 0000000180004c9a f   MSVCRT:dll_dllmain.obj
 0001:00003cd0       __scrt_is_nonwritable_in_current_image$filt$0 0000000180004cd0 f   MSVCRT:utility.obj
 0002:00000218       ?__scrt_initialize_tss_var@@3P6AHXZEA 0000000180005218     MSVCRT:thread_safe_statics.obj
 0002:00000340       ?opcLengths@@3QBEB         0000000180005340     libfollowref004.obj
 0002:00002300       GS_ExceptionPointers       0000000180007300     MSVCRT:gs_report.obj
 0002:000029b0       $unwind$fprintf            00000001800079b0     libfollowref004.obj
 0002:000029bc       $unwind$printf             00000001800079bc     libfollowref004.obj
 0002:000029c8       $unwind$?NewObject@JNIEnv_@@QEAAPEAV_jobject@@PEAV_jclass@@PEAU_jmethodID@@ZZ 00000001800079c8     libfollowref004.obj
 0002:000029c8       $unwind$nsk_lcomplain      00000001800079c8     libfollowref004.obj
 0002:000029c8       $unwind$nsk_ldisplay       00000001800079c8     libfollowref004.obj
 0002:000029d0       $unwind$nsk_jvmti_waitForSync 00000001800079d0     libfollowref004.obj
 0002:000029d0       $unwind$nsk_lvdisplay      00000001800079d0     libfollowref004.obj
 0002:000029d0       $unwind$_RTC_Initialize    00000001800079d0     MSVCRT:initsect.obj
 0002:000029d0       $unwind$_RTC_Terminate     00000001800079d0     MSVCRT:initsect.obj
 0002:000029d0       $unwind$?__scrt_initialize_thread_safe_statics@@YAHXZ 00000001800079d0     MSVCRT:thread_safe_statics.obj
 0002:000029dc       $unwind$nsk_complain       00000001800079dc     libfollowref004.obj
 0002:000029dc       $unwind$nsk_printf         00000001800079dc     libfollowref004.obj
 0002:000029e4       $unwind$nsk_lvcomplain     00000001800079e4     libfollowref004.obj
 0002:000029fc       $unwind$nsk_ltrace         00000001800079fc     libfollowref004.obj
 0002:000029fc       $unwind$__report_gsfailure 00000001800079fc     MSVCRT:gs_report.obj
 0002:00002a04       $unwind$nsk_lvtrace        0000000180007a04     libfollowref004.obj
 0002:00002a04       $unwind$stringPrimitiveValueCallback 0000000180007a04     libfollowref004.obj
 0002:00002a04       $unwind$__raise_securityfailure 0000000180007a04     MSVCRT:gs_report.obj
 0002:00002a04       $unwind$__scrt_initialize_crt 0000000180007a04     MSVCRT:utility.obj
 0002:00002a04       $unwind$__scrt_initialize_onexit_tables 0000000180007a04     MSVCRT:utility.obj
 0002:00002a04       $unwind$__scrt_release_startup_lock 0000000180007a04     MSVCRT:utility.obj
 0002:00002a04       $unwind$__scrt_uninitialize_crt 0000000180007a04     MSVCRT:utility.obj
 0002:00002a04       $unwind$_onexit            0000000180007a04     MSVCRT:utility.obj
 0002:00002a0c       $unwind$nsk_lverify        0000000180007a0c     libfollowref004.obj
 0002:00002a1c       $unwind$arrayPrimitiveValueCallback 0000000180007a1c     libfollowref004.obj
 0002:00002a1c       $unwind$nsk_vprintf        0000000180007a1c     libfollowref004.obj
 0002:00002a1c       $unwind$primitiveFieldCallback 0000000180007a1c     libfollowref004.obj
 0002:00002a2c       $unwind$?nsk_jni_lverify@@YAHHPEAUJNIEnv_@@HQEBDH1ZZ 0000000180007a2c     libfollowref004.obj
 0002:00002a40       $unwind$?nsk_jni_check_exception@@YAHPEAUJNIEnv_@@QEBDH@Z 0000000180007a40     libfollowref004.obj
 0002:00002a5c       $unwind$nsk_jvmti_parseOptions 0000000180007a5c     libfollowref004.obj
 0002:00002a78       $unwind$nsk_jvmti_createJVMTIEnv 0000000180007a78     libfollowref004.obj
 0002:00002a8c       $unwind$Java_nsk_jvmti_unit_FollowReferences_FollowRefObjects_resetTags 0000000180007a8c     libfollowref004.obj
 0002:00002a8c       $unwind$addRefToVerify     0000000180007a8c     libfollowref004.obj
 0002:00002a8c       $unwind$jvmti_FollowRefObject_init 0000000180007a8c     libfollowref004.obj
 0002:00002a8c       $unwind$nsk_jvmti_resetAgentData 0000000180007a8c     libfollowref004.obj
 0002:00002a8c       $unwind$nsk_jvmti_resumeSync 0000000180007a8c     libfollowref004.obj
 0002:00002a8c       $unwind$nsk_jvmti_setFailStatus 0000000180007a8c     libfollowref004.obj
 0002:00002a8c       $unwind$wrongArrayPrimitiveValueCallback 0000000180007a8c     libfollowref004.obj
 0002:00002a8c       $unwind$wrongHeapReferenceCallback 0000000180007a8c     libfollowref004.obj
 0002:00002a8c       $unwind$wrongPrimitiveFieldCallback 0000000180007a8c     libfollowref004.obj
 0002:00002a8c       $unwind$wrongStringPrimitiveValueCallback 0000000180007a8c     libfollowref004.obj
 0002:00002a8c       $unwind$__scrt_initialize_default_local_stdio_options 0000000180007a8c     MSVCRT:default_local_stdio_options.obj
 0002:00002a8c       $unwind$?dllmain_crt_dispatch@@YAHQEAUHINSTANCE__@@KQEAX@Z 0000000180007a8c     MSVCRT:dll_dllmain.obj
 0002:00002a8c       $unwind$DllMain            0000000180007a8c     MSVCRT:dll_dllmain_stub.obj
 0002:00002a8c       $unwind$__GSHandlerCheck   0000000180007a8c     MSVCRT:gshandler.obj
 0002:00002a8c       $unwind$?__scrt_uninitialize_thread_safe_statics@@YAXXZ 0000000180007a8c     MSVCRT:thread_safe_statics.obj
 0002:00002a8c       $unwind$__scrt_acquire_startup_lock 0000000180007a8c     MSVCRT:utility.obj
 0002:00002a8c       $unwind$__scrt_dllmain_after_initialize_c 0000000180007a8c     MSVCRT:utility.obj
 0002:00002a8c       $unwind$__scrt_dllmain_before_initialize_c 0000000180007a8c     MSVCRT:utility.obj
 0002:00002a8c       $unwind$__scrt_dllmain_crt_thread_attach 0000000180007a8c     MSVCRT:utility.obj
 0002:00002a8c       $unwind$__scrt_dllmain_crt_thread_detach 0000000180007a8c     MSVCRT:utility.obj
 0002:00002a8c       $unwind$__scrt_dllmain_uninitialize_c 0000000180007a8c     MSVCRT:utility.obj
 0002:00002a8c       $unwind$__scrt_dllmain_uninitialize_critical 0000000180007a8c     MSVCRT:utility.obj
 0002:00002a8c       $unwind$atexit             0000000180007a8c     MSVCRT:utility.obj
 0002:00002a94       $unwind$nsk_jvmti_lverify  0000000180007a94     libfollowref004.obj
 0002:00002aa8       $unwind$exitOnError        0000000180007aa8     libfollowref004.obj
 0002:00002ab8       $unwind$checkThatAllTagsVisited 0000000180007ab8     libfollowref004.obj
 0002:00002ab8       $unwind$check_option       0000000180007ab8     libfollowref004.obj
 0002:00002ab8       $unwind$_DllMainCRTStartup 0000000180007ab8     MSVCRT:dll_dllmain.obj
 0002:00002ac8       $unwind$Java_nsk_share_jvmti_ArgumentHandler_getAgentOptionsString 0000000180007ac8     libfollowref004.obj
 0002:00002adc       $unwind$Java_nsk_jvmti_unit_FollowReferences_FollowRefObjects_getTag 0000000180007adc     libfollowref004.obj
 0002:00002adc       $unwind$Java_nsk_share_jvmti_DebugeeClass_checkStatus 0000000180007adc     libfollowref004.obj
 0002:00002adc       $unwind$agentThreadWrapper 0000000180007adc     libfollowref004.obj
 0002:00002aec       $unwind$printHeapRefCallbackInfo 0000000180007aec     libfollowref004.obj
 0002:00002aec       $unwind$startAgentThreadWrapper 0000000180007aec     libfollowref004.obj
 0002:00002b08       $unwind$syncDebuggeeStatus 0000000180007b08     libfollowref004.obj
 0002:00002b08       $unwind$__scrt_dllmain_exception_filter 0000000180007b08     MSVCRT:utility.obj
 0002:00002b1c       $unwind$Java_nsk_share_jvmti_DebugeeClass_resetAgentData 0000000180007b1c     libfollowref004.obj
 0002:00002b24       $unwind$MA_checkStatus     0000000180007b24     libfollowref004.obj
 0002:00002b38       $unwind$markRefToVerify    0000000180007b38     libfollowref004.obj
 0002:00002b40       $unwind$checkUserData      0000000180007b40     libfollowref004.obj
 0002:00002b48       $unwind$Java_nsk_jvmti_unit_FollowReferences_FollowRefObjects_setTag 0000000180007b48     libfollowref004.obj
 0002:00002b60       $unwind$Java_nsk_jvmti_unit_FollowReferences_FollowRefObjects_addRefToVerify 0000000180007b60     libfollowref004.obj
 0002:00002b7c       $unwind$Agent_Initialize   0000000180007b7c     libfollowref004.obj
 0002:00002b98       $unwind$heapReferenceCallback 0000000180007b98     libfollowref004.obj
 0002:00002bb0       $unwind$createGlobalRefs   0000000180007bb0     libfollowref004.obj
 0002:00002bc8       $unwind$agentProc          0000000180007bc8     libfollowref004.obj
 0002:00002be4       $unwind$capture_previous_context 0000000180007be4     MSVCRT:gs_report.obj
 0002:00002bf0       $unwind$__GSHandlerCheckCommon 0000000180007bf0     MSVCRT:gshandler.obj
 0002:00002bf8       $xdatasym                  0000000180007bf8     MSVCRT:amdsecgs.obj
 0002:00002bfc       $unwind$?dllmain_crt_process_attach@@YAHQEAUHINSTANCE__@@QEAX@Z 0000000180007bfc     MSVCRT:dll_dllmain.obj
 0002:00002c38       $unwind$?fin$0@?0??dllmain_crt_process_attach@@YAHQEAUHINSTANCE__@@QEAX@Z@4HA 0000000180007c38     MSVCRT:dll_dllmain.obj
 0002:00002c38       $unwind$?fin$0@?0??dllmain_crt_process_detach@@YAH_N@Z@4HA 0000000180007c38     MSVCRT:dll_dllmain.obj
 0002:00002c38       $unwind$?fin$1@?0??dllmain_crt_process_detach@@YAH_N@Z@4HA 0000000180007c38     MSVCRT:dll_dllmain.obj
 0002:00002c40       $unwind$?dllmain_crt_process_detach@@YAH_N@Z 0000000180007c40     MSVCRT:dll_dllmain.obj
 0002:00002c94       $unwind$?dllmain_dispatch@@YAHQEAUHINSTANCE__@@KQEAX@Z 0000000180007c94     MSVCRT:dll_dllmain.obj
 0002:00002cbc       $unwind$?filt$0@?0??dllmain_dispatch@@YAHQEAUHINSTANCE__@@KQEAX@Z@4HA 0000000180007cbc     MSVCRT:dll_dllmain.obj
 0002:00002cc4       $unwind$__scrt_is_nonwritable_in_current_image 0000000180007cc4     MSVCRT:utility.obj
 0002:00002ce4       $unwind$__scrt_is_nonwritable_in_current_image$filt$0 0000000180007ce4     MSVCRT:utility.obj
 0002:00002cec       $unwind$__scrt_fastfail    0000000180007cec     MSVCRT:utility_desktop.obj
 0002:00002cfc       $unwind$__security_init_cookie 0000000180007cfc     MSVCRT:gs_support.obj
 0002:00002d08       $unwind$__isa_available_init 0000000180007d08     MSVCRT:cpu_disp.obj
 0002:00002d18       $xdatasym                  0000000180007d18     MSVCRT:guard_dispatch.obj
 0002:00002d20       $xdatasym                  0000000180007d20     MSVCRT:guard_xfg_dispatch.obj
 0002:00002d30       .edata                     0000000180007d30     followref004.exp
 0002:00002d58       rgpv                       0000000180007d58     followref004.exp
 0002:00002d90       rgszName                   0000000180007d90     followref004.exp
 0002:00002dc8       rgwOrd                     0000000180007dc8     followref004.exp
 0002:00002de4       szName                     0000000180007de4     followref004.exp
 0002:00002df5       $N00001                    0000000180007df5     followref004.exp
 0002:00002e04       $N00002                    0000000180007e04     followref004.exp
 0002:00002e11       $N00003                    0000000180007e11     followref004.exp
 0002:00002e56       $N00004                    0000000180007e56     followref004.exp
 0002:00002e93       $N00005                    0000000180007e93     followref004.exp
 0002:00002edb       $N00006                    0000000180007edb     followref004.exp
 0002:00002f1b       $N00007                    0000000180007f1b     followref004.exp
 0002:00002f58       $N00008                    0000000180007f58     followref004.exp
 0002:00002f93       $N00009                    0000000180007f93     followref004.exp
 0002:00002fc1       $N00010                    0000000180007fc1     followref004.exp
 0002:00002ff2       $N00011                    0000000180007ff2     followref004.exp
 0002:00003021       $N00012                    0000000180008021     followref004.exp
 0002:00003050       $N00013                    0000000180008050     followref004.exp
 0002:00003085       $N00014                    0000000180008085     followref004.exp
 0002:000034ea       .idata$6                   00000001800084ea     kernel32:KERNEL32.dll
 0002:0000354e       .idata$6                   000000018000854e     vcruntime:VCRUNTIME140.dll
 0002:000036e0       .idata$6                   00000001800086e0     ucrt:api-ms-win-crt-heap-l1-1-0.dll
 0002:00003700       .idata$6                   0000000180008700     ucrt:api-ms-win-crt-runtime-l1-1-0.dll
 0002:00003722       .idata$6                   0000000180008722     ucrt:api-ms-win-crt-convert-l1-1-0.dll
 0002:00003744       .idata$6                   0000000180008744     ucrt:api-ms-win-crt-stdio-l1-1-0.dll
 0002:00003764       .idata$6                   0000000180008764     ucrt:api-ms-win-crt-string-l1-1-0.dll
 0003:00000000       ?codeAttributeName@@3PEBDEB 0000000180009000     libfollowref004.obj
 0003:00000008       ?lineNumberAttributeName@@3PEBDEB 0000000180009008     libfollowref004.obj
 0003:00000010       ?localVarAttributeName@@3PEBDEB 0000000180009010     libfollowref004.obj
 0003:00000018       ?localVarTypeAttributeName@@3PEBDEB 0000000180009018     libfollowref004.obj
 0003:00000020       ?stackMapAttributeName@@3PEBDEB 0000000180009020     libfollowref004.obj
 0003:00000028       ?callBytes@@3PAEA          0000000180009028     libfollowref004.obj
 0003:0000002c       ?allocBytes@@3PAEA         000000018000902c     libfollowref004.obj
 0003:0001aad4       redefineAttempted          0000000180023ad4     libfollowref004.obj
 0003:0001aad8       nsk_context                0000000180023ad8     libfollowref004.obj
 0003:0001aae4       redefineSucceed            0000000180023ae4     libfollowref004.obj
 0003:0001aae8       agentFailed                0000000180023ae8     libfollowref004.obj
 0003:0001aaec       currentAgentStatus         0000000180023aec     libfollowref004.obj
 0003:0001aaf0       context                    0000000180023af0     libfollowref004.obj
 0003:0001aba8       agentThread                0000000180023ba8     libfollowref004.obj
 0003:0001abb0       agentThreadProc            0000000180023bb0     libfollowref004.obj
 0003:0001abb8       agentThreadArg             0000000180023bb8     libfollowref004.obj
 0003:0001abc0       agent_data                 0000000180023bc0     libfollowref004.obj
 0003:0001abd0       jvmti_env                  0000000180023bd0     libfollowref004.obj
 0003:0001abd8       jvm                        0000000180023bd8     libfollowref004.obj
 0003:0001abe0       jni_env                    0000000180023be0     libfollowref004.obj
 0003:0001abe8       checkStatus_func           0000000180023be8     libfollowref004.obj
 0003:0001abf0       ?codeAttributeIndex@@3GA   0000000180023bf0     libfollowref004.obj
 0003:0001abf4       ?lineNumberAttributeIndex@@3GA 0000000180023bf4     libfollowref004.obj
 0003:0001abf8       ?localVarAttributeIndex@@3GA 0000000180023bf8     libfollowref004.obj
 0003:0001abfc       ?localVarTypeAttributeIndex@@3GA 0000000180023bfc     libfollowref004.obj
 0003:0001ac00       ?stackMapAttributeIndex@@3GA 0000000180023c00     libfollowref004.obj
 0003:0001ac04       ?stackFrameOffset@@3GA     0000000180023c04     libfollowref004.obj
 0003:0001ac08       ?mode@@3HA                 0000000180023c08     libfollowref004.obj
 0003:0001ac0c       ?constantPoolSize@@3GA     0000000180023c0c     libfollowref004.obj
 0003:0001ac10       ?orig@@3PEBEEB             0000000180023c10     libfollowref004.obj
 0003:0001ac18       ?gen@@3PEAEEA              0000000180023c18     libfollowref004.obj
 0003:0001ac20       ?inputPos@@3PEAEEA         0000000180023c20     libfollowref004.obj
 0003:0001ac28       ?endPos@@3PEBEEB           0000000180023c28     libfollowref004.obj
 0003:0001ac30       ?genPos@@3PEAEEA           0000000180023c30     libfollowref004.obj
 0003:0001ac38       ?markPos@@3PEAEEA          0000000180023c38     libfollowref004.obj
 0003:0001ac40       ?constantPool@@3PEAPEADEA  0000000180023c40     libfollowref004.obj
 0003:0001ac48       ?constantPoolCount@@3GA    0000000180023c48     libfollowref004.obj
 0003:0001ac4c       ?zeroBytes@@3PAEA          0000000180023c4c     libfollowref004.obj
 0003:0001ac50       ?codeLength@@3IA           0000000180023c50     libfollowref004.obj
 0003:0001ac58       ?map@@3PEAIEA              0000000180023c58     libfollowref004.obj
 0003:0001ac60       ?widening@@3PEACEA         0000000180023c60     libfollowref004.obj
 0003:0001ac68       g_timeout                  0000000180023c68     libfollowref004.obj
 0003:0001ac70       g_jniGlobalRef             0000000180023c70     libfollowref004.obj
 0003:0001ac78       g_jniWeakGlobalRef         0000000180023c78     libfollowref004.obj
 0003:0001ac80       g_heapCallbacks            0000000180023c80     libfollowref004.obj
 0003:0001ad10       GS_ExceptionRecord         0000000180023d10     MSVCRT:gs_report.obj
 0003:0001adb0       GS_ContextRecord           0000000180023db0     MSVCRT:gs_report.obj
 0003:0001b280       ?g_tss_cv@@3U_RTL_CONDITION_VARIABLE@@A 0000000180024280     MSVCRT:thread_safe_statics.obj
 0003:0001b288       ?g_tss_event@@3PEAXEA      0000000180024288     MSVCRT:thread_safe_statics.obj
 0003:0001b290       ?g_tss_mutex@@3U_RTL_CRITICAL_SECTION@@A 0000000180024290     MSVCRT:thread_safe_statics.obj
 0003:0001b2b8       ?g_sleep_condition_variable_cs@@3P6AHPEAU_RTL_CONDITION_VARIABLE@@PEAU_RTL_CRITICAL_SECTION@@K@ZEA 00000001800242b8     MSVCRT:thread_safe_statics.obj
 0003:0001b2c0       ?g_wake_all_condition_variable@@3P6AXPEAU_RTL_CONDITION_VARIABLE@@@ZEA 00000001800242c0     MSVCRT:thread_safe_statics.obj
 0003:0001b2cc       ?__proc_attached@@3HA      00000001800242cc     MSVCRT:dll_dllmain.obj
 0003:0001b2e0       ?is_initialized_as_dll@@3_NA 00000001800242e0     MSVCRT:utility.obj
 0003:0001b2e1       ?module_local_atexit_table_initialized@@3_NA 00000001800242e1     MSVCRT:utility.obj
 0003:0001b2e8       ?module_local_atexit_table@@3U_onexit_table_t@@A 00000001800242e8     MSVCRT:utility.obj
 0003:0001b300       ?module_local_at_quick_exit_table@@3U_onexit_table_t@@A 0000000180024300     MSVCRT:utility.obj
